:100000000C94B1010C94CE010C94CE010C94CE0151
:100010000C94CE010C94CE010C94CE010C94CE0124
:100020000C94CE010C94CE010C9439250C940B2623
:100030000C94821F0C94CE010C94CE010C94CE0132
:100040000C94CE010C94CE010C94CE010C94CE01F4
:100050000C94CE010C940A200C94CE010C94CE0189
:100060000C94CE010C94CE010C94CE010C94CE01D4
:100070000C94CE010C94CE010C94CE010C94CE01C4
:100080000C94CE010C94CE010C94CE010C94CE01B4
:100090000C94CE010C94CE010C94CE010C94CE01A4
:1000A0000C94CE010C94CE010C94CE017E067E06FB
:1000B000AA06AA0612073007480848083B07D407D3
:1000C000E507E50778269F2697279F269727EB26A3
:1000D0000E279727652774271150AD00A800AC00A4
:1000E000AE00AB00125052080708500851084F08E4
:1000F0001350290029031B01060119011050150294
:100100004C00E0002C00130044454255473A20645F
:10011000697361626C65642E0A0044454255473A32
:1001200020656E61626C65642E0A000A002530321B
:1001300058006C65645F7461736B3A20004F6E65A4
:1001400073686F743A206163746976653A20256438
:100150000A000A0025303862003A20002530325863
:10016000000A722F632030313233343536370A00BB
:10017000290A002575002F002575005D28002564DB
:100180000020002564002000256400200025640074
:100190007C0025303258006D6F7573656B65792072
:1001A0005B62746E7C782079207620685D287265A9
:1001B000702F61636C293A205B000A0025303258A9
:1001C00020006B6579626F6172645F7265706F7237
:1001D000743A20005B735D005B575D005B535D000C
:1001E0005B525D005B445D005B435D000E036E008F
:1001F00065006F007000610064000000160372006B
:100200006F006F006B0069006500620077006F008F
:10021000790000000403090409025B00030100A047
:10022000FA09040000010301010009211101000184
:1002300022400007058103080001090401000103B1
:10024000000000092111010001227B000705820343
:10025000200001090402000203000000092111012D
:100260000001222200070583032000010705030384
:100270002000011201000200000008EDFE13091029
:1002800000010200010631FF0974A1010975150082
:1002900026FF009520750881020976150026FF00CB
:1002A000952075089102C005010902A10185020986
:1002B00001A10005091901290815002501950875F6
:1002C0000181020501093009311581257F950275EB
:1002D00008810609381581257F9501750881060575
:1002E0000C0A38021581257F950175088106C0C06A
:1002F00005010980A101850319012AB7001501260E
:10030000B700950175108100C0050C0901A1018598
:100310000419012AA002150126A002950175108179
:1003200000C005010906A101050719E029E715002C
:100330002501950875018102950175088101050760
:10034000190029FF150026FF009506750881000594
:10035000081901290595057501910295017503910B
:1003600001C011241FBECFEFDAE0DEBFCDBF11E028
:10037000A0E0B1E0EEEEF0E502C005900D92A43AE7
:10038000B107D9F722E0A4EAB1E001C01D92AA3773
:10039000B207E1F70E947B140C9475280C940000BE
:1003A000FF93EF93E091A401F091A501309709F03C
:1003B0000995EF91FF910895FC018591803011F02E
:1003C000EFDFFBCF0895FF27E0E230E247FF0CC0EC
:1003D000419597FF09C0EDE26095709580959095E5
:1003E000611D711D811D911D27FF02C0219530E304
:1003F00050E2AA27660F771F881F991FAA1FA4170C
:1004000010F0A41B63955A95A9F7AA3008F0A95FCC
:10041000A05DAF93F395611571058105910541F7D5
:10042000ED3211F4EF93F395F21718F43F93F3952F
:10043000FBCF8F91B5DFFA95E1F70895E991F99136
:100440008591803021F0853219F0AADFF9CF089527
:1004500020E0E89455915532C1F3503311F468947B
:1004600055915A3348F4505390F3220F022E220F25
:10047000220F200D250FF4CF0EF42195899199912B
:10048000533619F3533729F1533559F1BC018827F5
:100490009927E8945C3621F4899199916894559153
:1004A000543639F446EF7EF077FF0DC08FEF9FEFA3
:1004B0000AC055374AE039F0583540E121F052364C
:1004C00042E009F00895FF93EF937DDFEF91FF91F4
:1004D000B7CFFF93EF93FC0181918030B9F360DFD8
:1004E000FBCFFF93EF9368DFF1CFDF93CF93CDB7CF
:1004F000DEB72596A3DFCF91DF910895869A879A7C
:100500000C941B108E988F980895CF92DF92EF92E3
:10051000FF920E942D096B017C010E948F0480FFD5
:1005200002C08E9A01C08E9881FF02C08F9A01C0CE
:100530008F98C701B601FF90EF90DF90CF9008959C
:100540008E9A8F9A2FEF87EE93E021508040904053
:10055000E1F700C000008E988F982FEF87EE93E0B0
:10056000215080409040E1F700C000008E9A8F9AA1
:100570002FEF87EE93E0215080409040E1F700C0DC
:1005800000008E988F980C946513CF93C62F81111D
:1005900030C06091AD017091AE018091AF0190913A
:1005A000B0010E948F04813061F028F0823089F020
:1005B0008330B9F048C0CC2311F08BEA17C08CEA25
:1005C00015C0CC2319F08FE499E031C080E599E0A3
:1005D0002EC0CC2319F08CE191E029C08DE191E08F
:1005E00026C0CC2311F08CEF01C08BEF0E942C06AB
:1005F0002AC0813041F56091AD017091AE018091CA
:10060000AF019091B0010E948F04813061F028F019
:10061000823099F0833089F016C0CC2311F089EA3A
:10062000E5CF8AEAE3CFCC2329F08BE291E00E9468
:10063000880309C08BE296E0FACFCC2311F089EF52
:10064000D5CF8AEFD3CF81E0CF9108959C013A9521
:1006500021153F4130F5BC0166277270AC0144277B
:1006600054709C012227387094FF0FC090FF02C085
:1006700080E101C080E0672B09F08062452B09F022
:100680008064232B79F080680895892F8170672B0F
:1006900009F08260452B09F08460232B19F08860F3
:1006A000089580E00895CF93DF93EB010E94260325
:1006B000FE01DF91CF910994CF93DF93EC01805E2F
:1006C0009109089710F0209719F465E376E002C0CD
:1006D00060EC78E0CE010E9453038C2FDF91CF9124
:1006E0000C948B05CF93DF93EC010E94E105CE01C2
:1006F000805E9109089710F0209719F46CE376E07A
:1007000002C067EC78E0CE01DF91CF910C945303E7
:10071000CF93DF93EC010E945C03C933D10549F408
:100720002FEF87EE93E0215080409040E1F700C02A
:100730000000CE01DF91CF910C94720381E0089507
:1007400081E008950C94A00308950C94A4031F93D2
:10075000CF93DF9300D000D01F92CDB7DEB749838F
:100760005A836B833091A70189819A81311114C01A
:10077000662359F0222349F00E94910A182F682F0E
:1007800089819A810E943A0A03C00E94650A182F43
:1007900069817A81812F04C00E94910A69817A81DE
:1007A0000F900F900F900F900F90DF91CF911F91AE
:1007B0000C94DE11FC01262F4081518162817381EE
:1007C00084810C94A70381E00895CF93DF93EC011B
:1007D00060E00E94DA03BE01DF91CF910C94A50383
:1007E0000C94A0020C9463130E94E6080E948202FB
:1007F0002FEF84E39CE0215080409040E1F700C05F
:1008000000000C9430200F931F93CF93DF9300D000
:10081000CDB7DEB78C0161E00E94DA039A83898349
:10082000B801CE0101960E94041A882309F466C01B
:10083000B80189819A810E94A203882309F45EC0CD
:10084000B80189819A810E940E1E882309F456C03E
:10085000B80189819A810E949317882309F44EC0B8
:10086000B80189819A810E94D319882309F446C06E
:10087000F80182818823E9F189819A818F3D2CE5F5
:10088000920779F140F48115FCE59F0791F08130E2
:100890009C4591F02EC08C35EDE59E0741F18D35DC
:1008A000FDE59F0709F18B359D4519F50E94280F3D
:1008B00020C00E94F40322C080910F02182F1095CF
:1008C000117010FB80F980930F02112329F08AE147
:1008D00091E00E94DC0112C088E091E00E94DC01FE
:1008E0000EC00E94DC0F0AC00E941F0F02C00E94AF
:1008F0002B0FC8010E949E03182F01C010E0812F0A
:100900000F900F90DF91CF911F910F9108950E944A
:10091000631F0C9402050E9405050C94691FCF9279
:10092000DF92EF92FF926C01EE24FF24C114D104F8
:10093000E104F10421F0C701B60120E101C020E08B
:10094000C72ED82EE92EFF24C114D104E104F104EE
:1009500019F0285FC701B6016B017C0154E0F694E1
:10096000E794D794C7945A95D1F7C114D104E10400
:10097000F10419F02C5FC701B6016B017C0142E064
:10098000F694E794D794C7944A95D1F7C114D1044B
:10099000E104F10419F02E5FC701B601DC01CB01BF
:1009A000B695A79597958795892B8A2B8B2B09F060
:1009B0002F5F822FFF90EF90DF90CF900895829568
:1009C000982F937344E0949F900111248C7C86951A
:1009D0008695282B822F8575880F2A7A2695822B5B
:1009E000089508950C94F10481E008950C94F404A2
:1009F0000895CF93C82F0E94F2048C2F0E94F60412
:100A0000CF91089580E00C94F9040E946A1E0C9422
:100A1000F904CF930E946A1EC82F8091A601C817BF
:100A200041F1C093A60180910F0282FF1EC080FF9A
:100A300004C082E391E00E94DC0180910F0280FFFC
:100A40000CC01F92CF938DE291E09F938F930E94F1
:100A500075020F900F900F900F9080910F0280FF02
:100A600004C08BE291E00E94DC018C2FCF910C94AA
:100A7000F904CF910895CF93DF93CDB7DEB72B97CD
:100A80000FB6F894DEBF0FBECDBF4F83588769877E
:100A90007A878B8761110E94570E9E012F5F3F4F0F
:100AA00086E0F90111928A95E9F785E0FE01379613
:100AB000D90101900D928A95E1F789819A814C8143
:100AC0005D81452B31F09F3F31F491E08F3F19F468
:100AD00003C091E001C090E090FF09C049815A81B4
:100AE0006B817C818D819E810E94780D05C0C9013A
:100AF0000E94E3038111F2CF2B960FB6F894DEBF6C
:100B00000FBECDBFDF91CF910895FC01808191810F
:100B10000E94D30A0895CF93882309F450C0C82FA8
:100B20008CEF8C0F813AD0F46C2F80910201909160
:100B300003010E94051F882349F06C2F8091020158
:100B4000909103010E943D1F0E94790E6C2F8091AD
:100B50000201909103010E943B1F0CC080E28C0FA8
:100B6000883058F4C77081E001C0880FCA95EAF751
:100B70000E943A0ECF910C94790EEBE5EC0FE33026
:100B800040F4F0E0E95BFE4F808190E0CF910C945F
:100B9000CD1EE8E5EC0FE73150F4F0E0EE0FFF1F5B
:100BA000E75EFE4F80819181CF910C94E31ECD3E94
:100BB00030F08C2F0E940015CF910C94D215CF915C
:100BC0000895882389F19CEF980F913A40F4682F9B
:100BD00080910201909103010E943D1F0DC090E29F
:100BE000980F983058F4877091E001C0990F8A955A
:100BF000EAF7892F0E94400E0C94790E9BE5980F1E
:100C0000933020F480E090E00C94CD1E98E5980F8E
:100C1000973120F480E090E00C94E31E8D3E20F0AC
:100C20000E945B150C94D21508951F93CF93DF9308
:100C3000182FEB010E948B05209741F08FE99FE070
:100C40000197F1F700C000002197F6CF812FDF91C7
:100C5000CF911F910C94E105893319F060E070E0A9
:100C600002C060E570E00C941506882321F00E9414
:100C70003A0E0C94790E0895882321F00E94400EBC
:100C80000C94790E0895CF92DF92EF92FF920F931A
:100C90001F93CF93DF937C01D62FC72FFC011281C6
:100CA000058102950F700E94300E8823B9F0112340
:100CB000A9F08C2F807F803421F080E28D0F883066
:100CC00068F08091640282FD09C082E00E94D90E22
:100CD0000E94300E91E0D82ED92601C0D12CCC2E06
:100CE000C2948FE0C8228C2D90E08C30910508F0E2
:100CF000CFC1FC01EA5AFF4F0C94EA278C2F807F6A
:100D0000CF70882311F0C295C07F112399F0CC23B6
:100D100009F4AAC180E28D0F883010F0D11104C00F
:100D20008C2F0E943A0E03C08C2F0E944A0E0E9404
:100D3000790E9AC18D2F0E94E105CC2309F4A8C138
:100D400080E28D0F883038F1DD2329F18C2F0E944D
:100D5000500E24C08C2F807FCF70803211F0C2954E
:100D6000C07FDD2319F0D130A1F13DC08091640234
:100D700082FF17C0112349F0CC2329F08C2F0E9449
:100D80003A0E0E94790E80E070C180E00E94E10579
:100D9000CC2309F47DC18C2F0E94400E0E94790E55
:100DA00077C1112371F0002341F0013031F40E942A
:100DB0005A0E8C2B0E94620E6BC10E945A0E8C2B15
:100DC0001DC0002319F0013009F462C10E946F0EAA
:100DD00025C0112321F0033008F05AC10EC00230A3
:100DE00008F056C11BC0112361F0002331F0F70158
:100DF000858180FF39C18F7085838C2F0E943506D5
:100E000047C1002359F0D93309F03FC1FFEF07EE86
:100E100013E0F15000401040E1F735C18C2F0E94E3
:100E20003C0636C18C2F86958695837019F08130EB
:100E300061F02EC1112321F08D2F9C2F937002C0E1
:100E400080E090E00E94CD1E2BC1112321F08D2F58
:100E50009C2F937002C080E090E00E94E31E20C1AE
:100E60008D2F112319F00E94001502C00E945B15FE
:100E70000E94D21515C18C2F837009F047C0111143
:100E80000BC12D2F229526952770220F220F6D2F33
:100E90006F70862F90E0A0E0B0E0022E04C0880FB3
:100EA000991FAA1FBB1F0A94D2F7D4FF10C04FE0AE
:100EB00050E060E070E004C0440F551F661F771FCC
:100EC0002A95D2F7409550956095709503C040E003
:100ED00050E0BA01C695C695C3708A019B01082BE4
:100EE000192B2A2B3B2BC901B801C23049F058F409
:100EF000C13019F00E945209CFC00E944009CCC0F5
:100F00000E946409C9C00E943E09C6C0112319F09D
:100F10008C2F817001C08695882309F4BDC02D2FC8
:100F2000229526952770220F220F6D2F6F70862F26
:100F300090E0A0E0B0E0022E04C0880F991FAA1F25
:100F4000BB1F0A94D2F7D4FF10C04FE050E060E01E
:100F500070E004C0440F551F661F771F2A95D2F713
:100F6000409550956095709503C040E050E0BA01FF
:100F7000C695C695C3708A019B01082B192B2A2B95
:100F80003B2BC901B801C23049F058F4C13019F007
:100F90000E94150A81C00E94030A7EC00E94270A8F
:100FA0007BC00E94760978C0CF70112339F08C2F56
:100FB0000E949C098D2F0E9435066EC08D2F0E94C5
:100FC0003C068C2F0E94BD0967C0D23F21F128F456
:100FD000D03F41F0D13FC1F043C0D33F19F1D43FDE
:100FE00079F03EC0112341F0023008F051C08C2F3F
:100FF0008F710E94E2094CC0033008F049C0F7CF5E
:101000008091640282FF18C0112339F08C2F8F71F8
:101010000E949C093DC01123C9F38C2F8F710E943F
:10102000BD0936C0112329F08C2F8F710E948709CA
:101030002FC00E9482092CC0112349F0CF718C2F40
:101040000E949C0963E08C2F0E94BE0E21C081E0AB
:101050000E94D90E0230E0F082E00E94D90E18C042
:10106000112331F0002391F28D2F0E948B0510C0C7
:10107000002399F2D93349F41FEF27EE33E01150E2
:1010800020403040E1F700C000008D2F0E94E105B4
:1010900088EF8C0D843020F40E946A1E0E94F904AF
:1010A000DD20C9F00E942C0E80FD15C0F7011282D0
:1010B0000E94260E0E949C09C7010E948C080E9473
:1010C000260EDF91CF911F910F91FF90EF90DF904F
:1010D000CF900C94BD09DF91CF911F910F91FF909C
:1010E000EF90DF90CF9008950F931F93CF93DF93EE
:1010F000EC01688179818A810E94DE0A8C010E945C
:10110000390A0E942C09B801CE010E944306DF91E2
:10111000CF911F910F910895CF93DF93EC019881A8
:1011200089812B813C81232B31F08F3F31F481E089
:101130009F3F19F403C081E001C080E080FD1DC025
:10114000CE010E940304811110C00E94300E88233A
:10115000A1F08A81882389F08091640282FD0DC00C
:1011600082E0DF91CF910C94D90ECE010E947408D9
:10117000CE01DF91CF910C94E503DF91CF910895DB
:10118000882321F00E944A0E0C94790E089588233A
:1011900021F00E94500E0C94790E089580E090E0AA
:1011A0000E94CD1E80E090E00E94E31E0E94570E38
:1011B0000E94790E0E9485170C94D215809102012D
:1011C000909103010E943F1F0C94CE080E94470E8D
:1011D0000C94DE0892959F70963079F010F492503E
:1011E00001C09A50923068F4803F69F018F4883E4C
:1011F00040F409C0843F29F406C0883E20F0813FB6
:1012000011F080E0089581E00895FC0180819181D2
:101210000E94D30A0E94EA080895CF93DF9300D07A
:1012200000D01F92CDB7DEB70F900F900F900F90A8
:101230000F90DF91CF910895CF93DF9300D000D02E
:1012400000D0CDB7DEB726960FB6F894DEBF0FBE3E
:10125000CDBFDF91CF910895089508950C942D0985
:101260000C942E090E9430096093B1017093B20171
:101270008093B3019093B4010C94CE080C9432097E
:101280000F931F930091B1011091B2012091B3010E
:101290003091B401602B712B822B932B1F910F91F6
:1012A0000C9432090F931F930091B1011091B20178
:1012B0002091B3013091B4016023712382239323E1
:1012C0001F910F910C9432090F931F930091B1015C
:1012D0001091B2012091B3013091B40160277127C0
:1012E000822793271F910F910C9432090E94850247
:1012F0006093AD017093AE018093AF019093B00104
:101300000C94CE0860E070E0CB010C9476090F934A
:101310001F9341E050E060E070E08A019B0104C04F
:10132000000F111F221F331F8A95D2F7C901B80180
:101330001F910F910C9476090F931F9341E050E099
:1013400060E070E004C0440F551F661F771F8A9548
:10135000D2F78091AD019091AE01A091AF01B09113
:10136000B0018A019B01082B192B2A2B3B2BC901A9
:10137000B8011F910F910C9476090F931F9341E0D0
:1013800050E060E070E004C0440F551F661F771FF7
:101390008A95D2F740955095609570958091AD01F2
:1013A0009091AE01A091AF01B091B0018A019B0173
:1013B000082319232A233B23C901B8011F910F9148
:1013C0000C9476090F931F9341E050E060E070E0C9
:1013D00004C0440F551F661F771F8A95D2F780916E
:1013E000AD019091AE01A091AF01B091B0018A0121
:1013F0009B01082719272A273B27C901B8011F91FC
:101400000F910C9476090F931F930091AD011091E9
:10141000AE012091AF013091B001602B712B822B76
:10142000932B1F910F910C9476090F931F930091AA
:10143000AD011091AE012091AF013091B001602358
:101440007123822393231F910F910C9476090F939C
:101450001F930091AD011091AE012091AF01309129
:10146000B00160277127822793271F910F910C9459
:1014700076090895292F220F920F890FE82FE695FC
:10148000E695E695877051E001C0550F8A95EAF719
:1014900085E0E89FF0011124E855FE4F20E030E0A0
:1014A00070E04081CB01022E02C0969587950A9488
:1014B000E2F78170819584278523842781932F5FAC
:1014C0003F4F2530310569F70895292F220F920FDC
:1014D000890F682F669566956695982F977085E0B9
:1014E000689FB001112440E050E080E0FB01E40F70
:1014F000F51FE855FE4F208130E0092E02C03695D9
:1015000027950A94E2F721703327042E01C0220F99
:101510000A94EAF7822B4F5F5F4F4530510531F750
:101520000895BF92CF92DF92EF92FF920F931F9395
:10153000CF93DF938C01C090AD01D090AE01E090CD
:10154000AF01F090B0018091B1019091B201A091F2
:10155000B301B091B401C82AD92AEA2AFB2ACFE103
:10156000D0E0D701C6010C2E04C0B695A79597957B
:1015700087950A94D2F780FD04C0219790F7B12C8B
:1015800007C0BC2EB8018C2F0E94F4110197A9F35B
:101590008B2DDF91CF911F910F91FF90EF90DF90F6
:1015A000CF90BF900895CF93DF93EC010E94910AF2
:1015B000BE010E94F411DF91CF9108951F93CF9344
:1015C000DF93EB019091A701992321F0CB010E94B9
:1015D000D30A13C0882349F0CB010E94910A182F27
:1015E000682FCE010E943A0A04C0CB010E94650A0E
:1015F000182FBE01812F0E94F411DF91CF911F910E
:1016000008951F93CF93DF93C091B50116E08091A9
:10161000B601C81799F0D0E01C9FF0011D9FF00D96
:101620001124E954FE4F408151816281738184818C
:1016300095810E941C092196C770E9CFDF91CF9157
:101640001F9108954091E7015091E8016091E901EF
:101650007091EA018091EB019091EC010C941C09CE
:10166000EF92FF920F931F93CF93DF938091EC0142
:1016700082958F7009F065C08091E901882309F493
:1016800060C08091B501F090B6011091E701009122
:10169000E8016091EA017091EB0191E01F3F09F0D0
:1016A00090E0C0910001D0910101292F96E0E92E30
:1016B0008F1509F446C06115710521F00F3F21F027
:1016C00030E003C031E001C0322F90E030FD36C081
:1016D000E89EF001E99EF00D1124DF01A954BE4FF0
:1016E00011963C911197301329C03C91311326C0BB
:1016F00012963C911297311121C013964D915C9135
:101700001497461B570B4C175D07C0F48091EC01F2
:101710008F7080618093EC01E454FE4F80818F7064
:101720008061808387EE91E00E948C08DF91CF91E9
:101730001F910F91FF90EF900C94010B0196877011
:10174000B7CFDF91CF911F910F91FF90EF90089548
:101750009F92AF92BF92CF92DF92EF92FF920F9340
:101760001F93CF93DF93CDB7DEB761970FB6F89491
:10177000DEBF0FBECDBF8C0185E0F801DE011D96F6
:1017800001900D928A95E1F7D8011296EC90909114
:10179000E701E091E8012091EA013091EB01211588
:1017A000310531F0EF3F31F481E09F3F19F403C080
:1017B00081E001C080E0B82FB1709B2E80FD47C151
:1017C000D8014C9111965C9111971396AD90BC90F5
:1017D000149787EEC82E81E0D82EF090E901B5016C
:1017E000621B730B2091000130910101FF2009F46D
:1017F000D9C08091EC016217730708F095C0282FBB
:10180000207F09F052C05E1313C0491311C0FE2C93
:10181000E1100EC08F7080618093EC010E94220B5A
:10182000C6010E948C088091EC01F80185834DC1AE
:10183000AB2831F05F3F31F481E04F3F19F403C032
:1018400081E001C080E080FD03C081E08E2502C000
:1018500080E090E0F82FF170FF2E80FF1CC0809197
:10186000B5012091B60136E0821709F40BC190E072
:10187000389FF001399FF00D1124E954FE4F61812A
:10188000561306C06081461303C06281E61203C08E
:1018900001968770E9CFFE2CEE2009F416C18091E5
:1018A000EC0181608093EC0154C05E1306C04913C3
:1018B00004C0E11002C0F80199C0C8010E940509E6
:1018C000882361F1EE2051F12091EC01822F829565
:1018D0008F7090E0029774F08091E7019091E80199
:1018E00098878F831986BB86AA862C87CE01079698
:1018F0000E948C0886E0F801A7EEB1E001900D92FD
:101900008A95E1F70E94300B0E94220B0AC05E17F5
:1019100011F1C8010E94050981112CC0C8010E9463
:101920008C08FF24F394D1C0282F207F81F77A2DD3
:10193000B98AA88A6E2D89890E940D0987EE91E0E7
:101940000E948C0886E0D6011D928A95E9F70E94D4
:10195000220BF12CBAC04913DCCFE110DACFF80129
:101960008583C8010E948C0886E0D6011D928A9565
:10197000E9F7ABC0EE2091F22091EC01822F829525
:101980008F7090E002970CF4B5CF8091E7019091B1
:10199000E8019A8389831B82BD82AC822E83CE01AB
:1019A0000196A6CF6217730708F044C0FE2CEE2004
:1019B00009F4B4CF5E1330C049132EC02091EC015E
:1019C00020FD21C0822F82958F70482F50E0411555
:1019D0005105C9F0F80125834F30510541F08F5F63
:1019E000982F9295907F822F8F70892B8583C801C5
:1019F0000E948C0886E0F801A7EEB1E001900D92FC
:101A00008A95E1F73CC086E0F801A7EEB1E00190CD
:101A10000D928A95E1F759C0C8010E94050981110C
:101A200069CF8091EC0181608093EC01C8010E9434
:101A30008C084BC07A2DB98AA88A6E2D89890E949C
:101A40000D0986E0D6011D928A95E9F718C0EE20AF
:101A500009F464CFC8010E940509F82E882309F40F
:101A60005DCF86E0F801A7EEB1E001900D928A9576
:101A7000E1F787EE91E00E9485050E94300B0E94FD
:101A8000220B23C04D875E878D859E850E94D30AD9
:101A9000292F22952F70223028F49F7039F0811160
:101AA00005C00BC0243028F49F7049F4805E883054
:101AB00020F0C8010E948C089F2CF92C06C0D80188
:101AC00015969C91907F91F7F8CF8F2D61960FB668
:101AD000F894DEBF0FBECDBFDF91CF911F910F9164
:101AE000FF90EF90DF90CF90BF90AF909F900895C0
:101AF0001F93CF93DF93CDB7DEB72C970FB6F89433
:101B0000DEBF0FBECDBF4F83588769877A878B872B
:101B10009C87CE0107960E94A80B8823D1F09F8155
:101B200088852A853B85232B31F08F3F31F481E076
:101B30009F3F19F403C081E001C080E080FD47C0F1
:101B40004F81588569857A858B859C850E941C0903
:101B50003EC086E0FE013796DE01119601900D929F
:101B60008A95E1F7FF81E8856A857B8561157105B6
:101B700031F0EF3F31F481E0FF3F19F403C081E021
:101B800001C080E080FD23C02091B60130E0C90192
:101B90000196877099274091B50150E08417950709
:101BA000F1F1F983EA837D836C8396E0929FD00103
:101BB000939FB00D1124A954BE4FFE0131960190A0
:101BC0000D929A95E1F78093B6010E94010B16E001
:101BD0008091B5019091B601891771F1189FC001EC
:101BE000112489549E4F0E94A80B882329F1E0916B
:101BF000B5011E9FF0011124E954FE4F408151812F
:101C000062817381848195810E941C098091B50154
:101C100090E00196877099278093B501D9CF0E94F3
:101C2000E6081092B6011092B501E7EEF1E086E009
:101C3000DF011D928A95E9F72C960FB6F894DEBF66
:101C40000FBECDBFDF91CF911F9108958091F50117
:101C500085958595859508958091F50187700895FE
:101C60009091F501977081E009F480E008958091EA
:101C70000002089590910002892B8093000208953C
:101C8000809590910002892380930002089510921C
:101C9000000208959091FF01892B8093FF01089520
:101CA00080959091FF0189238093FF010895109200
:101CB000FF0108958091F601089508950C945D0E3A
:101CC0000C945E0E9091640292FD08C09091F60112
:101CD000981721F08093F6010C94600E089580917E
:101CE000F601882329F01092F60180E00C94600E32
:101CF0000895CF93DF93E0910201F0910301809169
:101D000000028083E0910201F091030190818091B3
:101D1000FF01892B80838091F601882381F0E09177
:101D20000201F09103019081892B8083809102014F
:101D3000909103010E94F91E81110E946F0EC091C3
:101D40000201D091030148E050E06DEE71E0CE0158
:101D50000E942628892B69F088E0FE01ADEEB1E0F3
:101D600001900D928A95E1F7CE01DF91CF910C940D
:101D7000761EDF91CF9108950C945D0E90916402D0
:101D800092FD10C098E0899F90011124262B20938A
:101D9000F5010E949C098091F501859585958595B1
:101DA0000C94BC0E0C949C091092F50180E00C94EC
:101DB000BC0E2091F501809582238093F501982F28
:101DC000977099F430E0482F082E000C550B24171B
:101DD000350759F09091640292FD07C0859585956D
:101DE00085950E94BD090C94D40E0895CF939091CF
:101DF000640292FB222720F92817F9F0C82F892FB7
:101E0000C0FB82F980936402809163029091640226
:101E10000E94580F82E00E94D90E80910F0280FF2D
:101E20000CC01F92CF938DE391E09F938F930E94FC
:101E300075020F900F900F900F90CF9108958091A1
:101E4000640282FB882780F991E089270C94F60EC2
:101E500081E00C94F60E80E00C94F60E6FEF7FEFAD
:101E600080E090E00C945F2880E090E00E943B28A6
:101E700021E0893E9E4F09F020E0822F089582E004
:101E800090E00C94332883E090E00C943328CF93B7
:101E900084E090E00E943328C82F82E290E00E9404
:101EA00033282C2F30E0A901582BCA01CF91089577
:101EB000CF93C92F682F84E090E00E9441286C2FB7
:101EC00082E290E0CF910C944128AB01BC018FE0FD
:101ED00090E00C945328AB01BC0183E190E00C949A
:101EE000532860E070E0CB010C946B0F60E070E071
:101EF000CB010E94650F0C94710F69EE7EEF80E0BC
:101F000090E00E945F2860E082E090E00E9441281B
:101F100060E083E090E00E9441281092B1011092AD
:101F2000B2011092B3011092B40160E084E090E03D
:101F30000E94412860E082E290E00E94412860E037
:101F400085E090E00E94412860E086E090E00E94F9
:101F500041286FEF87E090E00E94412840E050E088
:101F6000BA0188E090E00E94532860E08DE090E0A4
:101F70000E94412840E050E0BA0188E190E00E94D0
:101F8000532860E087E190E00E94412840E050E063
:101F9000BA018CE190E00E94532860E070E080E29A
:101FA00090E00E945F2840E050E0BA0188E190E0B4
:101FB0000E9453280C94760F0C947D0F682F8EE0AE
:101FC00090E00C9441280E94EF1F60930B027093E5
:101FD0000C0280930D0290930E026093070270939F
:101FE00008028093090290930A0208950E94EF1F4D
:101FF00060930B0270930C0280930D0290930E027B
:10200000609303027093040280930502909306028A
:10201000089585B7806885BF85B7806885BF0895B6
:1020200081E008950C94101008950C9414100C94F1
:1020300014100C9417100C9414100C9414100E948B
:10204000091084E192E20E94601E0E941D100C940F
:102050007E020E9415100C9414100E94E8120C9439
:10206000F8040E94DA1F0E94F1130E942D100E94B2
:10207000E4180C9419108F929F92AF92BF92CF9256
:10208000DF92EF92FF920F931F93CF93DF93CDB721
:10209000DEB72A970FB6F894DEBF0FBECDBF0E9401
:1020A0000014982E81110E94E30F81E0A82E82E097
:1020B000B82E00E010E0802E802F0E940C13D82E46
:1020C000F501C1905F01C826B1F40F5F1F4F0230C8
:1020D000110589F78FEF89838A831B820E94E31F92
:1020E0008160782F9D838C8349815A816B818D819A
:1020F0000E943B052FC080910F0281FD0E941213A8
:10210000E12CFF24F3948C2D8F21F1F00E9412100A
:10211000882399F0EE828F82DF2081E009F480E04D
:1021200088870E94E31F8160782F9A8789874E8174
:102130005F8168858A850E943B05F801EF5FFD4F4E
:102140008081F826F08206C0E394FF0CF3E0EF12E2
:10215000DACFBBCF81E0911001C080E02A960FB6A4
:10216000F894DEBF0FBECDBFDF91CF911F910F91CD
:10217000FF90EF90DF90CF90BF90AF909F908F90A7
:1021800008950E943B100E94361981110E94F60F9B
:102190000E9472160C940905CF93DF930E94F911E7
:1021A000EC01811521E5920708F045C0811530E565
:1021B000930708F094C0883E910528F5803E91056C
:1021C00008F0F8C0883A910570F4853A910508F056
:1021D0007CC08130910509F475C008F4E8C004970B
:1021E00008F0E8C0E4C08F3B910508F0E0C0C85A91
:1021F000D0E0CC0FDD1FC65BDE4F0990D881C02D2B
:10220000CE019464D8C0811540E2940758F481153A
:1022100051E0950708F0CEC08D3E910508F4C7C087
:102220009065C9C0C11580E4D80708F4C0C0DF704C
:10223000CE01906AC0C0811525E59207A8F48115EA
:1022400034E5930708F095C0811543E5940708F03D
:102250007BC0811552E5950708F061C0D82FCC27C7
:10226000CE01816F906AA7C0C11589E5D807A0F497
:10227000C11528E5D20708F082C0C11536E5D3079D
:1022800008F095C08C2F0E948D128F7190E0D82F8E
:10229000CC27CE0190628FC0C1154AE5D40708F45F
:1022A00074C0CE0190568115904208F080C08D2FE9
:1022B0008F710E948D12DD27D0628F71AE01582B75
:1022C000CA0179C081E090E076C0C55AD0E0C85814
:1022D000DE4F8881C82FD0E0CE0190646CC074E0DE
:1022E000969587957A95E1F7282F23703C2F3370C8
:1022F00081E090E002C0880F991F3A95E2F79C6850
:10230000AC01522B9A019C2F9F709695969550E2A6
:10231000959FE0011124C9018C2B9D2B4CC083702B
:10232000992721E030E002C0220F331F8A95E2F79F
:102330009C2F9695969580E2989FE0011124C22BE0
:10234000D32BCE019C6837C08370992721E030E001
:1023500002C0220F331F8A95E2F79C2F969596951F
:1023600040E2949FE0011124C22BD32BCE019A6846
:1023700022C0D82FCC27CE01846F906A1CC0DC2FDE
:10238000CC27CE01806F906A16C08C2F8F700E9470
:102390008D1294E0D695C7959A95E1F7CF70D0E06D
:1023A000DC2FCC27D0699E01282BC90104C080E016
:1023B00090E001C0CE01DF91CF910895272F30E04A
:1023C000F901EE0FFF1F2E0F3F1FF90196E0899FC5
:1023D000E00DF11D1124E60FF11DEE0FFF1FE85275
:1023E000FF4F8591949108950E94DE110E94CC10B8
:1023F00008958238910569F1B0F48133910509F4AB
:102400006DC048F48932910509F463C08A329105A0
:1024100009F469C008958533910509F455C08933DD
:102420009105B9F00895833E910569F138F4803E35
:102430009105B1F0823E910509F10895863E91051E
:10244000A9F1873E9105B9F1843E910509F064C078
:1024500023C02091630220FD4FC021FD4DC008958F
:102460008091630280FD44C08091640280FF44C07B
:102470008091630284FD42C083EE4DC0809163026F
:1024800082FF38C0F5CF8091630282FD33C0809116
:10249000640280FD31C0ECCF8091640281FF32C0C4
:1024A0008091630284FD2AC087EE35C0809163026B
:1024B00083FF26C0F5CF8091630283FD21C0809108
:1024C000640281FD1FC0ECCF8091630285FD1CC0BA
:1024D0001DC08091630285FD19C016C08091630202
:1024E00086FD16C017C08091630286FD13C010C020
:1024F00089E311C082EE0FC080EE0DC080E00BC0FA
:1025000086EE09C084EE07C089E205C085E303C0FA
:102510008AE201C081E390E008959091630292FF06
:102520000DC0282F2871283019F4877F846006C0D9
:10253000282F2471243011F48B7F886093FF0DC005
:10254000282F2871283119F4877E846106C0282F2E
:102550002471243111F48B7E88612091640220FF64
:102560000DC0382F3871383019F4877F816006C06C
:10257000382F3171313011F48E7F886021FF0DC00A
:10258000282F2871283119F4877E816106C0282FF1
:102590002171213111F48E7E886194FD877E08952A
:1025A0000C942E0F0E9400148FE39CE90197F1F721
:1025B00000C000000E94001480E00E940C1380FF05
:1025C00004C00E94D0120C94302008950C94D212B2
:1025D0000E94340F811102C00E94DC0F0E943F0F45
:1025E00080930F020E94470F9093640280936302CE
:1025F0000E94E6120E94430F682F70E080E090E096
:102600000E943E096091AD017091AE018091AF01D1
:102610009091B0010C948502E82FF0E0E959FD4F4C
:1026200080810895CF92DF92EF92FF920F931F93D4
:10263000CF93DF9381E691E00E94DC0187E6E82EEC
:1026400082E0F82EC0E0D0E09CE5C92E91E0D92EC2
:1026500004E511E0DF93CF93DF92CF920E947502E1
:1026600089E591E00E94DC01F70181917F010E94E0
:10267000DF041F928F931F930F930E94750282E5D0
:1026800091E00E94DC0121968DB79EB708960FB6A7
:10269000F8949EBF0FBE8DBFC230D105D9F6DF9131
:1026A000CF911F910F91FF90EF90DF90CF90089501
:1026B00080EA8A95F1F7089500C008950C945813A4
:1026C00008950C9460130C9461130C946013F894A7
:1026D000E82FE295EF70F0E031A1282F2F7081E014
:1026E00090E001C0880F2A95EAF7982F90959323E0
:1026F00091A392A1892B82A37894089584EF0E94DC
:10270000671385EF0E94671383E30E94671382E3D8
:102710000E94671386E30C946713CF92DF92EF92C7
:10272000FF920F931F93CF93DF938C01C62FD0E0BE
:10273000CE0182589E4F7C01FC0190819F3F09F49D
:1027400047C0D62EF894E92FE295EF70F0E081A112
:102750009F7021E030E001C0220F9A95EAF7822BAA
:1027600081A382A12095282322A378940E945C1340
:10277000EBE7F1E04EE751E031E0C12C21912F3F32
:1027800089F0A22FA295AF70B0E090968C9190E066
:102790002F7002C0959587952A95E2F780FD02C0BB
:1027A000832F01C080E0C82A330F4E175F0731F72F
:1027B000F70180818F3F11F00E94671361E0C11023
:1027C00001C060E08D2D0E945E13C00FD11FC88232
:1027D000DF91CF911F910F91FF90EF90DF90CF90FD
:1027E00008950E947E131092680210926702109260
:1027F00066021092650282E00E9438140C94F00385
:102800001F93CF93DF9300D0CDB7DEB71A82198222
:1028100060E0CE0101960E948D1361E0CE01019629
:102820000E948D1342E050E0BE016F5F7F4F85E64E
:1028300092E00E94262811E0009709F410E0892B0D
:1028400031F089819A819093660280936502212FED
:1028500042E067E672E085E692E00E9439140E9449
:10286000F203812F0F900F90DF91CF911F91089568
:102870000895FF920F931F93CF93DF938C01F62E51
:10288000D72FC42F222349F081E0809312020E94A7
:10289000E31F90931102809310028091120288230B
:1028A000C1F080911002909111020E94FB1F0597C8
:1028B00080F0EF2DFD2FD8014C2F50E0CD01801B73
:1028C000910B841795071CF48D918193F7CF10928B
:1028D0001202DF91CF911F910F91FF9008950E94F6
:1028E00090220E9431100C949C220E94A0220E94EF
:1028F000C1100C94BE220E94811F0E9477220E9468
:102900001F100E946F140E9475140E942910FBCFA3
:102910008091190280FF06C06091090170E0660F86
:10292000771F26C081FF04C06091090184E005C0C3
:1029300082FF07C06091090188E0689FB0011124FF
:1029400017C0909118029923D1F060910801961751
:1029500088F72091090188E0289F90011124929F17
:10296000A001939F500D112470E0CA010E94D62748
:102970006038710540F46115710519F406C068E00E
:1029800070E0862F08958FE7089581E00895809183
:10299000190280FF08C06091050170E07595679588
:1029A0007595679521C081FF06C06091050170E0B3
:1029B0007595679519C082FF04C06091050170E0AC
:1029C00010C090911702992399F060910401961715
:1029D000A0F780910501899FC001112470E00E9439
:1029E000D6276038710540F46115710519F406C0E9
:1029F00061E070E0862F08958FE7089581E00895E3
:102A00008D3E21F40E948814819504C08E3E29F4E5
:102A10000E94881480931D0208958F3E21F40E9425
:102A20008814819504C0803F29F40E948814809303
:102A30001C020895893F19F40E94C71405C08A3FFB
:102A400031F40E94C714819580931E0208958B3F34
:102A500021F40E94C714819504C08C3F29F40E9480
:102A6000C71480931F0208959FE0980F983078F460
:102A700021E030E0A90102C0440F551F9A95E2F70A
:102A8000CA0190911B02892B80931B0208958D3FF0
:102A900021F48091190281600BC08E3F21F4809156
:102AA0001902826005C08F3F29F480911902846069
:102AB0008093190208958D3E39F490911D0297FF7D
:102AC00035C010921D0259C08E3E29F490911D020E
:102AD0001916BCF32BC090911C028F3E29F497FF6E
:102AE00025C010921C0249C0803F19F41916CCF37E
:102AF0001DC090911E02893F29F41916BCF4109252
:102B00001E023BC08A3F19F497FF10C0F8CF8B3FDD
:102B100039F490911F0297FF09C010921F022DC037
:102B20008C3F21F490911F021916BCF39FE0980F7F
:102B3000983080F421E030E0A90102C0440F551F15
:102B40009A95E2F7CA01809590911B0289238093A0
:102B50001B0213C08D3F21F4809119028E7F0BC0A0
:102B60008E3F21F4809119028D7F05C08F3F29F49B
:102B7000809119028B7F8093190280911C02811130
:102B800006C080911D02811102C01092180280912E
:102B90001E02811106C080911F02811102C0109295
:102BA0001702089580910F0283FF7EC087E991E0AC
:102BB0000E94DC0180911B021F928F9382E991E0B9
:102BC0009F938F930E94750280E991E00E94DC013F
:102BD00080911C02282F082E000C330B3F938F93FB
:102BE0008DE891E09F938F930E9475028BE891E0AE
:102BF0000E94DC0180911D02282F082E000C330B4F
:102C00003F938F9388E891E09F938F930E94750282
:102C100086E891E00E94DC0180911E02282F082E98
:102C2000000C330B3F938F9383E891E09F938F9336
:102C30000E94750281E891E00E94DC0180911F02F0
:102C4000282F082E000C330B3F938F938EE791E0D3
:102C50009F938F930E9475028BE791E00E94DC01A5
:102C6000809118021F928F9388E791E09F938F9332
:102C70000E94750286E791E00E94DC0180911902B2
:102C80001F928F9383E791E09F938F930E94750229
:102C900080E791E00E94DC018DB79EB74C960FB69D
:102CA000F8949EBF0FBE8DBF0E94E31F20911C02AF
:102CB000211104C020911D02222321F090931602BD
:102CC0008093150220911E02211104C020911F0241
:102CD000222321F090931402809313028AE192E060
:102CE0000C94BF1EEF92FF920F931F93CF93DF932D
:102CF00000D000D000D0CDB7DEB786E0EAE1F2E048
:102D0000DE01119601900D928A95E1F7E0901C0288
:102D1000F0901D0200911E0210911F0210921C02E1
:102D200010921D0210921E0210921F02E11003C0A9
:102D3000FF2009F45DC080911502909116020E9457
:102D4000FB1FAC0190911802992339F020910A01E0
:102D500030E02417350758F04BC020910B018AE072
:102D6000289F900111242417350718F041C09F3F78
:102D700019F09F5F90931802EE2061F00E94881472
:102D80001E1414F09FEF01C091E0989F902D112424
:102D900090931C02FF2061F00E9488141F1414F00D
:102DA0009FEF01C091E0989F902D112490931D02F8
:102DB00030911C023323E1F020911D022223C1F047
:102DC00045EB3403C0011124992319F090931C02A0
:102DD00003C081E080931C0235EB2303C001112462
:102DE000992319F090931D0203C081E080931D0286
:102DF000011103C0112309F45DC080911302909169
:102E000014020E94FB1FAC0190911702992339F024
:102E10002091060130E02417350758F04BC020916F
:102E200007018AE0289F900111242417350718F024
:102E300041C09F3F19F09F5F90931702002361F0FC
:102E40000E94C714101614F09FEF01C091E0989FE4
:102E5000902D112490931E02112361F00E94C7143B
:102E6000111614F09FEF01C091E0989F902D11244E
:102E700090931F0230911E023323E1F020911F0234
:102E80002223C1F045EB3403C0011124992319F02A
:102E900090931E0203C081E080931E0235EB230352
:102EA000C0011124992319F090931F0203C081E0FF
:102EB00080931F0280911C0281110BC080911D0222
:102EC000811107C080911E02811103C080911F02F1
:102ED00081110E94D215EB82FC820D831E8386E055
:102EE000FE013196AAE1B2E001900D928A95E1F7D8
:102EF00026960FB6F894DEBF0FBECDBFDF91CF91FF
:102F00001F910F91FF90EF900895EAE1F2E086E0C3
:102F1000DF011D928A95E9F71092180210921702AC
:102F2000109219020895CF93DF93EC01FB01828187
:102F3000882309F43CC1C430FDE5DF0760F4CB3FD2
:102F40009CE5D90788F49E0122503C452431310587
:102F500008F02EC109C0C236EDE5DE0729F0C63AF9
:102F6000FDE5DF0709F024C10E94470F909364023A
:102F700080936302C1318CE5D80709F4C6C008F01C
:102F800042C0C930ECE5DE0709F49BC000F5C5304E
:102F90008CE5D80709F485C078F4C330ECE5DE078A
:102FA00009F478C008F07AC0C230DC4509F0F5C0F9
:102FB000809163028160EFC0C7309CE5D90709F4B6
:102FC00078C008F07AC0809163028061E4C0CD309F
:102FD000FCE5DF0709F487C058F4CB309CE5D9073E
:102FE00009F479C008F07BC08091630288606FC0EB
:102FF000CF30FCE5DF0709F480C008F082C0809183
:103000006302877FC8C0CE3F9CE5D90709F471C031
:1030100000F5C531FCE5DF0709F485C068F4C3316C
:103020009CE5D90709F475C008F095C00E94E60830
:10303000809163028F77AFC0CC3FFCE5DF07A9F139
:1030400008F054C0CB3FDC4509F0A7C08091640272
:1030500040C0C230EDE5DE0709F489C058F4C1155F
:103060008DE5D80709F45AC008F069C08091640260
:1030700082602FC0C236EDE5DE0709F47CC0C63A97
:10308000FDE5DF0709F481C0C330DD4509F085C0E7
:1030900080E06EC08091630282607DC08091630297
:1030A00016C080916302886076C08091640282605D
:1030B0004FC08091630280626EC080916302806421
:1030C0006AC00E94E60880916302806864C08460E0
:1030D00062C081603DC0809163028E7F5CC0809140
:1030E00063028D7F58C08091630216C08091640294
:1030F00018C0809164028D7F2BC0809163028F7E07
:103100004AC0809163028F7D46C0809163028F7BAD
:1031100042C080916302877F8B7F3DC080916402B3
:103120008D7F8E7F15C08091630282FB222720F95C
:1031300091E0922790FB82F990FB83F92CC080915B
:103140006402982F909591708E7F892B90FB81F966
:103150008093640222C00E94E6088091630287FB8C
:10316000222720F991E0922790FB87F914C081E093
:103170000E94DE0F12C08091630284FB222720F997
:1031800091E0922790FB84F906C080916302982F0A
:10319000909590FB80F980936302809163029091F7
:1031A00064020E94580F0E94E60880E001C081E09E
:1031B000DF91CF9108958FE891E00197F1F700C07A
:1031C000000008950C94C502CF93DF93A2E9B1E00B
:1031D000C0E9D1E021E030E071E0A439B70759F14E
:1031E0008D91E82FE295EF70F0E041A18F70B90169
:1031F00002C0660F771F8A95E2F7CB01962F909554
:10320000942391A392A1892B82A38991E82FE2951F
:10321000EF70F0E041A18F70B90102C0660F771F17
:103220008A95E2F7CB01962F9095942391A392A1D2
:10323000892B82A3D1CF0E94DB1889B1869581703A
:10324000489902C090E001C092E0892B809324024B
:1032500089B182958170369902C090E001C092E0F8
:10326000892B80932502DF91CF9108954F925F9231
:103270006F927F928F929F92AF92BF92CF92DF9286
:10328000EF92FF920F931F93CF93DF9304E212E02C
:1032900082E9C82E81E0D82E90E9E92E91E0F92E3E
:1032A00022E2822E22E0922EC0E2D2E05801512C7E
:1032B000412C34E0632E712CD501ED915D014E2F30
:1032C000440F440FF60121916F01E22FE295EF7058
:1032D000F0E080A190E02F7002C0959587952A9527
:1032E000E2F781709927D7015D917D01E52FE29585
:1032F000EF70F0E020A130E05F7002C035952795B7
:103300005A95E2F7F901E170FF2720FF02C0E2E0E1
:10331000F0E0E82BF92BE42BD801ED938D01EF7051
:10332000F0E0E058FE4F9081F4018081890F8083A6
:1033300084304CF088818F5F888360E0852D0E9407
:10334000E21821E001C020E0D4018C918D3F44F4CB
:1033500088818150888361E0852D0E94E21821E0F8
:10336000F4018081082E000C990BB3010E94D6272E
:10337000D4018D934D01422A53942196B2E05B1201
:103380009BCF842DDF91CF911F910F91FF90EF90F4
:10339000DF90CF90BF90AF909F908F907F906F9075
:1033A0005F904F900895CF93DF9386319C4541F510
:1033B000EB010E94370E982F8A81209102013091F3
:1033C0000301882379F09A7A81E009F480E0809300
:1033D0002602911102C069E201C065E3C9010E94A1
:1033E0003B1F0AC080912602811102C069E201C020
:1033F00065E3C9010E943D1F0E94790E80E001C073
:1034000081E0DF91CF9108958F929F92AF92BF920A
:10341000CF92DF92EF92FF920F931F93CF93DF93A0
:103420007C01DC01ED91FC91CF01815095458F3FEE
:10343000910510F4B5E5FB27DB011296CC91CC2366
:1034400009F4B4C2EF3FF10579F070F0EB32FD45BD
:1034500019F01092270260C39091270281E089271A
:1034600080932702A0E059C3A0912702AA2309F460
:10347000EBC010922702E03CF10540F4E038F10582
:1034800008F073C0E034F105D0F505C0EF3FF10559
:1034900009F008F4A0C021E030E040E050E060E036
:1034A00070E080E090E00E2F0E94F027B09128029B
:1034B0002B2BB09129023B2BB0912A024B2BB091C0
:1034C0002B025B2BB0912C026B2BB0912D027B2B2E
:1034D000B0912E028B2BB0912F029B2B20932802B0
:1034E0003093290240932A0250932B0260932C02BE
:1034F00070932D0280932E0290932F02A1C021E0A1
:1035000030E040E050E060E070E080E090E08F016B
:10351000005411090E94F027B09130022B2BB0917A
:1035200031023B2BB09132024B2BB09133025B2B1B
:10353000B09134026B2BB09135027B2BB0913602E7
:103540008B2BB09137029B2B2093300230933102AA
:1035500040933202509333026093340270933502E9
:1035600080933602909337026BC021E030E040E058
:1035700050E060E070E080E090E08F0100581109B9
:103580000E94F027B09138022B2BB09139023B2BCF
:10359000B0913A024B2BB0913B025B2BB0913C02B5
:1035A0006B2BB0913D027B2BB0913E028B2BB091E7
:1035B0003F029B2B209338023093390240933A020A
:1035C00050933B0260933C0270933D0280933E0215
:1035D00090933F0235C021E030E040E050E060E0F1
:1035E00070E080E090E08F01005C11090E94F027FC
:1035F000B09140022B2BB09141023B2BB091420283
:103600004B2BB09143025B2BB09144026B2BB091DA
:1036100045027B2BB09146028B2BB09147029B2B2E
:103620002093400230934102409342025093430260
:103630006093440270934502809346029093470240
:10364000E701F983E88369C2E034F105D0F4A09082
:103650002802B0902902C0902A02D0902B02E0905C
:103660002C02F0902D02B0912E0210912F0221E039
:1036700030E040E050E060E070E080E090E00E2F4D
:103680005DC0E038F105E8F4A0903002B09031025E
:10369000C0903202D0903302E0903402F0903502B4
:1036A000B09136021091370221E030E040E050E066
:1036B00060E070E080E090E04F01D0E48D1A910866
:1036C0003CC0E03CF105E8F4A0903802B09039022B
:1036D000C0903A02D0903B02E0903C02F0903D0254
:1036E000B0913E0210913F0221E030E040E050E016
:1036F00060E070E080E090E04F01D0E88D1A910822
:103700001CC0A0904002B0904102C0904202D090F4
:103710004302E0904402F0904502B09146021091BD
:10372000470221E030E040E050E060E070E080E0FF
:1037300090E04F01D0EC8D1A9108082D0E94F027DF
:10374000A222B322C422D522E622F722B8231923CB
:1037500021E030E040E050E060E070E080E090E0A8
:10376000E034F105A0F04F01E038F10520F4D0E499
:103770008D1A91080AC0E03CF10520F4D0E88D1ABA
:10378000910803C0D0EC8D1A9108082D01C00E2FAE
:103790000E94F0270B2F0E94092809F0BDC1E03CD0
:1037A000F10548F4E038F10508F084C0E034F10593
:1037B00008F042C005C0EF3FF10509F008F4B8C0B9
:1037C00021E030E040E050E060E070E080E090E038
:1037D0000E2F0E94F02720953095409550956095CA
:1037E000709580959095E09128022E23E091290212
:1037F0003E23E0912A024E23E0912B025E23E091CA
:103800002C026E23E0912D027E23E0912E028E2366
:10381000E0912F029E2320932802309329024093A7
:103820002A0250932B0260932C0270932D028093F6
:103830002E0290932F0271C18F010054110921E0D3
:1038400030E040E050E060E070E080E090E00E9416
:10385000F02720953095409550956095709580950E
:103860009095E09130022E23E09131023E23E091C9
:1038700032024E23E09133025E23E09134026E2344
:10388000E09135027E23E09136028E23E0913702EB
:103890009E232093300230933102409332025093A2
:1038A0003302609334027093350280933602909312
:1038B000370233C18F010058110921E030E040E0A8
:1038C00050E060E070E080E090E00E94F0272095FA
:1038D0003095409550956095709580959095E091C4
:1038E00038022E23E09139023E23E0913A024E2322
:1038F000E0913B025E23E0913C026E23E0913D02A9
:103900007E23E0913E028E23E0913F029E2320938E
:1039100038023093390240933A0250933B0260934D
:103920003C0270933D0280933E0290933F02F5C0AB
:103930008F01005C110921E030E040E050E060E0E0
:1039400070E080E090E00E94F0272095309540954F
:1039500050956095709580959095E09140022E234A
:10396000E09141023E23E09142024E23E091430266
:103970005E23E09144026E23E09145027E23E091B4
:1039800046028E23E09147029E232093400230930B
:103990004102409342025093430260934402709369
:1039A00045028093460290934702B7C0EF3FF1056E
:1039B00011F008F0AEC0E034F105D0F4C090280258
:1039C000D0902902E0902A02F0902B0210912C0254
:1039D000C0912D02B0912E02A0912F0221E030E083
:1039E00040E050E060E070E080E090E00E2F5DC0CD
:1039F000E038F105E8F4C0903002D0903102E09058
:103A00003202F090330210913402C0913502B0912D
:103A10003602A091370221E030E040E050E060E063
:103A200070E080E090E05F01D0E4AD1AB1083CC0E6
:103A3000E03CF105E8F4C0903802D0903902E09003
:103A40003A02F0903B0210913C02C0913D02B091CD
:103A50003E02A0913F0221E030E040E050E060E013
:103A600070E080E090E05F01D0E8AD1AB1081CC0C2
:103A7000C0904002D0904102E0904202F090430298
:103A800010914402C0914502B0914602A0914702B4
:103A900021E030E040E050E060E070E080E090E065
:103AA0005F01D0ECAD1AB1080A2D0E94F027A22EBA
:103AB000AC20B32EBD20C42ECE20D52EDF20E62E86
:103AC000E122F72EFC22B823192F1A23E034F10546
:103AD00070F0E038F10518F4E054F10908C0E03C5A
:103AE000F10518F4E058F10902C0E05CF10921E0A9
:103AF00030E040E050E060E070E080E090E00E2FC9
:103B00000E94F027A1E00B2F0E94092819F4A0E0E1
:103B100001C0A1E0A17001C0AC2F8A2FDF91CF912D
:103B20001F910F91FF90EF90DF90CF90BF90AF90DB
:103B30009F908F9008950F931F93CF93DF93C42F7F
:103B4000D22FFC0182818823C9F040934A020E944F
:103B5000E31F909349028093480280E28C0F8830E3
:103B600008F057C0C77081E001C0880FCA95EAF716
:103B7000DF91CF911F910F910C94350680914A02ED
:103B8000481330C080914802909149020E94FB1F67
:103B9000883C910538F510E21D0FCD17B9F080E291
:103BA0008C0F883040F4C77081E001C0880FCA953F
:103BB000EAF70E943C06183028F581E09D2F9770A7
:103BC00001C0880F9A95EAF70E943506802F0E945F
:103BD0002C061830F0F4D77081E001C0880FDA9518
:103BE000EAF70AC080E28C0F883098F4C77081E051
:103BF00001C0880FCA95EAF7DF91CF911F910F910D
:103C00000C943C06802FDF91CF911F910F910C9463
:103C10002C06DF91CF911F910F9108950F939C0176
:103C2000CB01243F4CE5340731F188F4293DFCE514
:103C30003F07D9F02A3D4CE5340779F1283D3C4552
:103C4000A9F506E221EE41EE68ED7CE52BC0263FAA
:103C5000FCE53F07E1F0A8F0273F3C4539F507E2D6
:103C600025EE46EE67EF7CE51DC007E225EE45EE4A
:103C700069ED7CE517C006E221EE40EE64EF7CE5DD
:103C800011C007E225EE44EE65EF7CE50BC006E2CD
:103C900021EE42EE66EF7CE505C008E221E045EE4C
:103CA0006AED7CE50E949B1D80E008C0FC018281DA
:103CB000882319F010924A0201C081E00F91089503
:103CC0009093A5018093A40108959093500280934E
:103CD0004F020895E0914F02F0915002309721F089
:103CE0000190F081E02D099480E00895EF92FF9219
:103CF0000F931F93CF93DF93E0914F02F091500207
:103D00003097B1F18C010280F381E02D099580910B
:103D10000F0282FF2DC080FF04C082EC91E00E9460
:103D2000DC01E80118E08CEBE82E81E0F82E8091B0
:103D30000F0280FF0BC088811F928F93FF92EF923A
:103D40000E9475020F900F900F900F9011502196C6
:103D50001111EDCF80910F0280FF0AC08AEB91E034
:103D6000DF91CF911F910F91FF90EF900C94DC01A8
:103D7000DF91CF911F910F91FF90EF900895E09107
:103D80004F02F0915002309739F022E0DC012C9381
:103D90000480F581E02D0994089520914D02309121
:103DA0004E022817390771F090934E0280934D020E
:103DB000E0914F02F0915002309721F00680F78198
:103DC000E02D0994089520914B0230914C02281760
:103DD000390771F090934C0280934B02E0914F02AF
:103DE000F0915002309721F00084F185E02D099484
:103DF0000895FC01329697E080E0915029F02191DE
:103E00002223D9F38F5FF9CF0895662349F0FC018F
:103E1000329608962191621729F0E817F907D1F731
:103E200080E0089581E008959C01FC0132969FEFA7
:103E300080E04191461789F09F3F19F4411101C07C
:103E4000982F8F5F8630A9F79F3F39F0F901E90F6E
:103E5000F11D97FDFA956283089508959C012A5FEC
:103E60003F4FFC014281461301C012820196821726
:103E70009307B9F708950C94141F0C942E1F029603
:103E800026E0FC0111922A95E9F7089508950C9413
:103E9000461F83E0809351020C94471F811102C09A
:103EA00081E001C082E0809351020C94471F0C9482
:103EB0004E1F81E0809351020C94471F0C94591FB0
:103EC00008950C94601F0C94611F0C94601F0C9457
:103ED000601F0C94601F0E94671F0E9400140E94C4
:103EE000651F80E00E940C13811108C081E00E94D0
:103EF0000C1391E0811103C090E001C091E0892F83
:103F0000089508951F920F920FB60F9211248F9368
:103F10009F93AF93BF9380915202811113C0809100
:103F2000690290916A02A0916B02B0916C02419675
:103F3000A11DB11D8093690290936A02A0936B0248
:103F4000B0936C02BF91AF919F918F910F900FBE74
:103F50000F901F90189580917102843031F10E946A
:103F600087041092520220E488E190E00FB6F894A2
:103F7000A895809360000FBE2093600083B7817F77
:103F8000846083BF83B7816083BF7894889583B74B
:103F90008E7F83BF0FB6F894A895809160008861EA
:103FA00080936000109260000FBE08950E94E608A2
:103FB0000C948B0482E084BD93E095BD9AEF97BD8D
:103FC00080936E0008952FB7F894809169029091C4
:103FD0006A02A0916B02B0916C022FBF08952FB7B7
:103FE000F8946091690270916A0280916B029091DD
:103FF0006C022FBF08959C014FB7F894809169021D
:1040000090916A02A0916B02B0916C024FBF821B2B
:10401000930B089578941F920F920FB60F9211246C
:104020008F939F93AF93BF938091690290916A029F
:10403000A0916B02B0916C020196A11DB11D8093FD
:10404000690290936A02A0936B02B0936C02BF91D5
:10405000AF919F918F910F900FBE0F901F90189569
:1040600087E797E790930108809300089AE088E13A
:104070000FB6F894A895809360000FBE90936000EF
:10408000FFCF809161020895089522E02093E90016
:104090002FEF3091E800215035FD06C035ED3A95FF
:1040A000F1F700002111F5CF2091E80025FF0BC0AA
:1040B00040E050E066E070E00E942D238091E8002F
:1040C0008E778093E8000895CF93DF9321E02093CB
:1040D000E9002FEF3091E800215035FD06C035EDA5
:1040E0003A95F1F700002111F5CF2091E80025FF66
:1040F00014C0EC0140E050E068E070E00E942D2325
:104100008091E8008E778093E80088E0FE01A9E5C1
:10411000B2E001900D928A95E1F7DF91CF91089579
:1041200080935502709357026093560280917102FA
:10413000843001F582E08093E9008FEF9091E800F0
:10414000815095FD06C095ED9A95F1F7000081111B
:10415000F5CF8091E80085FF0DC040E050E063E0BE
:1041600070E085E592E00E942D238091E8008E7733
:104170008093E8000895BC0184E00C949020BC0179
:1041800083E00C94902088EE91E00E94DC01809105
:104190007002811109C00E94BE240E941B258091DB
:1041A000E20084608093E200089584EE91E00E9432
:1041B000DC0110927002089580EE91E00E94DC0113
:1041C0000C945E1F8CED91E00E94DC0160916D0209
:1041D00081E0611101C080E00C94491F88ED91E0FD
:1041E0000E94DC019091710281E0943009F080E03E
:1041F00060916D020C944E1F209154022F5F822F0C
:1042000062E30E94CA27992319F02093540208956B
:104210001092540280915802882371F180917102AA
:10422000843041F58091E9008F702091EC00922F4D
:10423000917020FD90E8892B93E09093E900909194
:10424000EB0090FF14C09091EE0097FF10C090918A
:10425000E80095FF03C01092F100F9CF9091E800BB
:1042600090FF05C09091E8009E779093E8008F70D2
:104270008093E90010925802089542E061EC81E0D9
:104280000E94372442E261EC82E00E94372442E23D
:1042900061EC83E00E9437249091710281E09430B8
:1042A00009F080E060916D020C94571F80917302B9
:1042B000833009F461C030F4813071F0823009F448
:1042C0009AC008958A3009F486C08B3009F46CC016
:1042D000893009F0A8C020C080917202813A09F0AB
:1042E000A2C08091E800877F8093E80080917602E9
:1042F00090917702892B21F468E089E592E003C070
:1043000060E080E090E070E00E9478238091E80017
:104310008B778093E800089580917202813209F0D2
:1043200082C08091760290917702029708F07BC05C
:104330008091E800877F8093E8008091E80082FD0B
:1043400005C0809171028111F8CF6DC02091F300FA
:104350008091F20090E0922B029731F48091F1006D
:10436000813011F0863021F48091F1008093610258
:104370008091E8008B7753C080917202813A09F0F6
:1043800052C08091760290917702892B09F04BC040
:104390008091E800877F8093E8008091E80080FFAB
:1043A000FCCF8091180136C0809172028132D9F51C
:1043B0008091760290917702892BA9F58091E8008F
:1043C000877F8093E8000E946C2480917402809320
:1043D00018010C94E60880917202813221F58091D7
:1043E000E800877F8093E8000E946C24809175022A
:1043F00080936202089580917202813AA1F48091C3
:10440000E800877F8093E8008091E80080FFFCCF80
:10441000809162028093F1008091E8008E77809312
:10442000E8000C946C2408959FB7F89410925802F9
:104430009FBF90917102943009F057C09091E900AC
:104440009F703091EC00232F217030FD20E8922BDB
:1044500023E02093E9002091EB0020FF43C020914E
:10446000EE0027FF3FC020915302222321F020912C
:10447000E80025FF37C01092530226E03091E80093
:1044800035FD15C030917102343061F53091EB008B
:1044900035FD28C0215021F481E08093530222C0D1
:1044A000EFE9FFE03197F1F700C00000E7CF80931C
:1044B000F1008091E80085FD0AC08091E80080FF4E
:1044C000FCCF8091E8008E778093E80006C08FB71C
:1044D000F89421E0209358028FBF9F709093E900D9
:1044E00080E008959F709093E9008FEF089584B75E
:1044F000877F84BF0FB6F894A8958091600088618B
:1045000080936000109260000FBE90E080E80FB6CC
:10451000F89480936100909361000FBE0C94591F32
:104520000E94BE240E941B25E2EEF0E080818460A0
:10453000808378940C94AF278CE091E00C94651EF6
:10454000809171028530C9F484ED91E00E94DC0114
:1045500080917102853079F40E94AB1F80916F02C7
:104560008823B1F30E946B1F882391F30E941723C5
:104570000E94E608EDCF0C94D61F089508950C9480
:10458000C122292F332723303105C9F060F42130AF
:10459000310581F02230310509F041C08BE590E012
:1045A00028E132E040C021323105E1F0223231050C
:1045B00031F135C082E190E023E732E034C0992741
:1045C0008130910549F028F0029749F5ECEEF1E0D1
:1045D00005C0E4E1F2E002C0ECEFF1E0849190E08C
:1045E0009F0121C063307105D0F4660F771FFB0176
:1045F000E356FE4F2081318189E090E014C06330A2
:10460000710568F4FB01EE0FFF1FE956FE4F208194
:104610003181FB01EC56FE4F808190E004C080E0C8
:1046200090E020E030E0FA0131832083089580E1BA
:1046300089BD82E189BD09B400FEFDCF8091D8001B
:104640008F7D8093D8008091E00082608093E000AD
:104650008091E00081FDFCCF0895CF92DF92EF9230
:10466000FF920F931F93CF93DF93EC018B017A019D
:104670000E948B24811133C0E114F10439F0F70159
:1046800080819181081B190BC80FD91FC12CD12C17
:104690000115110519F18091E80085FD16C0809182
:1046A000E8008E778093E800E114F10449F0F70107
:1046B00080819181C80ED91ED182C08285E00FC051
:1046C0000E948B24882321F30AC089918093F100F2
:1046D00001501109FFEFCF1ADF0ADACF80E0DF9136
:1046E000CF911F910F91FF90EF90DF90CF900895A1
:1046F00020917802309179022617370748F061152A
:10470000710539F42091E8002E772093E80001C06C
:10471000B901FC0120E06115710579F18091710208
:104720008823F1F18530F1F18091E80083FD3CC0F0
:104730008091E80082FD2EC08091E80080FFEBCFE1
:104740002091F3008091F20090E0922B61157105A9
:1047500051F08830910538F421912093F100615097
:1047600071090196F3CF21E0089709F020E08091CC
:10477000E8008E778093E800CECF2111CFCF0AC01A
:1047800080917102882361F0853061F08091E800AA
:1047900083FD0AC08091E80082FFF2CF80E0089597
:1047A00082E0089583E0089581E0089520917802E1
:1047B000309179022617370748F06115710539F4F1
:1047C0002091E8002E772093E80001C0B901FC0198
:1047D00020E06115710591F180917102882309F43F
:1047E00040C0853009F43FC08091E80083FD3DC0A2
:1047F0008091E80082FD2FC08091E80080FFE9CF22
:104800002091F3008091F20090E0922B61157105E8
:1048100059F08830910540F424912093F1003196AD
:10482000615071090196F2CF21E0089709F020E06C
:104830008091E8008E778093E800CBCF2111CCCF18
:104840000AC080917102882361F0853061F0809107
:10485000E80083FD0AC08091E80082FFF2CF80E08B
:10486000089582E0089583E0089581E00895982FE7
:10487000973068F59093E900981739F07091EC0043
:104880002091ED005091F00003C0242F762F50E0CE
:1048900021FD02C09F5FECCF3091EB003E7F309353
:1048A000EB003091ED003D7F3093ED003091EB0057
:1048B00031603093EB007093EC002093ED00509347
:1048C000F0002091EE0027FDE5CF80E008958F7085
:1048D0008093E90081E008958091720287FF11C002
:1048E0008091E80082FD05C0809171028111F8CFAE
:1048F00011C08091E8008B770BC0809171028823F2
:1049000049F08091E80080FFF8CF8091E8008E7731
:104910008093E80008952091E4003091E50095E649
:104920004091EC00842F817040FF23C08091E8000B
:1049300080FD1DC080917102882399F0853099F027
:104940008091EB0085FD11C04091E4005091E5009D
:104950002417350729F3915011F09A01E1CF84E033
:10496000089582E0089583E0089581E0089580E04D
:1049700008954091E80042FFDDCF08950E942C2564
:104980000E943425E0EEF0E0808181608083E8EDD4
:10499000F0E080818F77808319BCA7EDB0E08C9127
:1049A0008E7F8C9380818F7E808310927002089519
:1049B0000F931F93CF93DF930E942C250E943425E1
:1049C000C8EDD0E088818F7788838881806888836C
:1049D00088818F7D888319BC1092710210926D02BC
:1049E00010926F0210926E0200EE10E0F8018081CA
:1049F0008B7F808388818160888342E060E080E0F3
:104A00000E943724E1EEF0E080818E7F8083E2EE29
:104A1000F0E0808181608083808188608083F801FC
:104A200080818E7F8083888180618883DF91CF91B0
:104A30001F910F910895E8EDF0E080818F7E8083D3
:104A4000E7EDF0E080818160808384E082BF81E0D7
:104A5000809370020C94D824E8EDF0E080818E7F82
:104A600080831092E20008951092DA001092E10023
:104A700008951F920F920FB60F9211242F933F9318
:104A80004F935F936F937F938F939F93AF93BF9356
:104A9000EF93FF938091E10082FF0BC08091E200D1
:104AA00082FF07C08091E1008B7F8093E1000E942C
:104AB000FC208091DA0080FF1FC08091D80080FF29
:104AC0001BC08091DA008E7F8093DA008091D9003C
:104AD00080FF0DC080E189BD82E189BD09B400FE7F
:104AE000FDCF81E0809371020E94C32005C019BCF4
:104AF000109271020E94D5208091E10080FF19C0C0
:104B00008091E20080FF15C08091E2008E7F80934B
:104B1000E2008091E20080618093E2008091D80001
:104B200080628093D80019BC85E0809371020E9456
:104B3000E2208091E10084FF30C08091E20084FF98
:104B40002CC080E189BD82E189BD09B400FEFDCFA2
:104B50008091D8008F7D8093D8008091E1008F7E76
:104B60008093E1008091E2008F7E8093E20080914B
:104B7000E20081608093E20080916D02882311F051
:104B800084E007C08091E30087FD02C081E001C09E
:104B900083E0809371020E94EE208091E10083FF08
:104BA00029C08091E20083FF25C08091E100877FCA
:104BB0008093E10082E08093710210926D028091F7
:104BC000E1008E7F8093E1008091E2008E7F8093F0
:104BD000E2008091E20080618093E20042E060E0C8
:104BE00080E00E9437248091F00088608093F0007C
:104BF0000E94DC20FF91EF91BF91AF919F918F9127
:104C00007F916F915F914F913F912F910F900FBEC8
:104C10000F901F9018951F920F920FB60F921124AC
:104C20002F933F934F935F936F937F938F939F93B4
:104C3000AF93BF93CF93DF93EF93FF93C091E900BE
:104C4000CF708091EC00D82FD17080FDD0E8109209
:104C5000E9008091F000877F8093F00078940E94B3
:104C60004F261092E9008091F00088608093F00058
:104C7000CD2BCF70C093E900FF91EF91DF91CF91E1
:104C8000BF91AF919F918F917F916F915F914F9164
:104C90003F912F910F900FBE0F901F9018951F936B
:104CA000CF93DF93CDB7DEB7AA970FB6F894DEBFE8
:104CB0000FBECDBFE2E7F2E08091F100819322E0E8
:104CC000EA37F207C9F70E9456218091E80083FF76
:104CD0002EC18091720290917302492F50E04A30A8
:104CE000510508F024C1FA01EE59FF4F0C94EA2750
:104CF000803821F0823809F01AC108C080916E0214
:104D000090916F02992389F082600FC080917602A2
:104D10008F70873008F00BC18093E9008091EB0021
:104D200085FB882780F91092E9009091E800977F31
:104D30009093E8008093F1001092F100D1C0282FE9
:104D40002D7F09F0F4C0882319F0823061F0EFC0A4
:104D500080917402813009F0EAC0933009F080E05C
:104D600080936F022EC08091740281112AC08091BD
:104D700076028F702FEF280F263008F0D8C080936E
:104D8000E9002091EB0020FF1CC0933021F48091BA
:104D9000EB00806214C09091EB0090619093EB0067
:104DA00021E030E0A90102C0440F551F8A95E2F7C7
:104DB0004093EA001092EA008091EB0088608093B3
:104DC000EB001092E9008091E800877F8093E80073
:104DD0000E946C24ACC08111AAC0109174021F778C
:104DE0008091E3008078812B8093E3008091E8003C
:104DF000877F8093E8000E946C248091E80080FF08
:104E0000FCCF8091E30080688093E300111102C021
:104E100082E001C083E08093710289C080588230B3
:104E200008F085C080917402909175028C3D53E02A
:104E3000950779F583E08A838AE289834FB7F894EE
:104E4000DE01139620E03EE051E2E32FF0E05093C4
:104E50005700E49120FF03C0E295EF703F5FEF70D1
:104E60008E2F90E0EA3010F0C79601C0C0968D9367
:104E70009D932F5F243149F74FBF8091E800877FD2
:104E80008093E8006AE270E0CE0101960E947823E8
:104E900016C06091760270917702AE014F5F5F4F4E
:104EA0000E94BF22BC01892B09F441C09091E80007
:104EB000977F9093E80089819A810E94D623809100
:104EC000E8008B778093E80032C0803881F58091CC
:104ED000E800877F8093E80080916D028093F10065
:104EE0008091E8008E7772CF811121C08091740289
:104EF0009091750299270297D4F48091E800877FFA
:104F00008093E8008091740280936D020E946C246B
:104F100080916D02811106C08091E30087FD02C07F
:104F200081E001C084E0809371020E943D21809164
:104F3000E80083FF0AC08091E800877F8093E80043
:104F40008091EB0080628093EB00AA960FB6F894F4
:104F5000DEBF0FBECDBFDF91CF911F910895CF93DC
:104F6000809171028823A1F0C091E900CF709091E7
:104F7000EC00892F817090FD80E8C82B1092E90029
:104F80008091E80083FD0E944F26CF70C093E90016
:104F9000CF910895991B79E004C0991F961708F0E6
:104FA000961B881F7A95C9F78095089597FB072E61
:104FB00016F4009407D077FD09D00E94122807FC50
:104FC00005D03EF4909581959F4F08957095619519
:104FD0007F4F0895EE0FFF1F0590F491E02D099487
:104FE0000F93083090F0982F872F762F652F542F2E
:104FF000432F322F22270850F4CF220F331F441F94
:10500000551F661F771F881F991F0A95B2F70F91CA
:1050100008952A153B054C055D056E057F05800743
:1050200091070895AA1BBB1B51E107C0AA1FBB1F14
:10503000A617B70710F0A61BB70B881F991F5A9524
:10504000A9F780959095BC01CD010895FB01DC0185
:1050500004C08D910190801921F441505040C8F74F
:10506000881B990B0895F999FECF92BD81BDF89ADE
:10507000992780B50895A8E1B0E042E050E00C9493
:105080006728262FF999FECF92BD81BDF89A019726
:1050900000B4021639F01FBA20BD0FB6F894FA9A80
:1050A000F99A0FBE08950396272F0E9442280E9466
:1050B0004128252F0E944228242F0C944228019633
:1050C000272F0E9442280C944128DC01CB01FC01CF
:1050D000F999FECF06C0F2BDE1BDF89A319600B451
:0E50E0000D9241505040B8F70895F894FFCF5C
:1050EE00C800F701280850011E0A1401412064204F
:1050FE004520BF20BB20442001E200E900EA00B5B4
:10510E0000B600B700CD008301CC008A0192019455
:10511E00012102230224022502260227022A02B3BB
:10512E0000B4006F007000818283E200E900EA00A3
:10513E00B500B600B700CD008301CC008A01920104
:10514E0094012102230224022502260227022A02AA
:10515E00B300B4006F007000818283333236F4F5F1
:10516E0000FF0100010000FFFF0000010001FF0031
:10517E0090669194407B222203A70285022A024365
:04518E00025C0200BD
:00000001FF
